:020000040000FA
:100000000C94F6050C94B01C0C94891C0C941E06E0
:100010000C941E060C941E060C941E060C941E06D0
:100020000C941E060C94D71C0C941E060C941E06F1
:100030000C941E060C941E060C941E060C941E06B0
:100040000C943F1C0C941E060C941E060C941E0669
:100050000C941E060C941E060C941E060C941E0690
:100060000C94491D0C941E0620002F00204F46546E
:100070003A004F6666200020002B004356310020D6
:10008000002B0043563200204D4F443A004F666625
:1000900020003025200020524E443A004F66662052
:1000A00000435600204D4F443A00494E542000452D
:1000B0005854313620004558542D4220004558549C
:1000C0003234200020434C4B3A0078002F004F463A
:1000D0004600312F31360042454154005050514EB8
:1000E000002032340062706D002062706D0020626A
:1000F000706D2000200000000000003E5B4F5B3E62
:100100003E6B4F6B3E1C3E7C3E1C183C7E3C181CDC
:10011000577D571C1C5E7F5E1C00183C1800FFE7D3
:10012000C3E7FF0018241800FFE7DBE7FF30483A79
:10013000060E2629792926407F050507407F0525DB
:100140003F5A3CE73C5A7F3E1C1C08081C1C3E7F63
:1001500014227F22145F5F005F5F06097F017F002A
:100160006689956A606060606094A2FFA29408044A
:100170007E040810207E201008082A1C08081C2A6B
:1001800008081E101010100C1E0C1E0C30383E38C3
:1001900030060E3E0E06000000000000005F00006A
:1001A0000007000700147F147F14242A7F2A1223DB
:1001B0001308646236495620500008070300001CEB
:1001C0002241000041221C002A1C7F1C2A08083EF4
:1001D0000808008070300008080808080000606007
:1001E0000020100804023E5149453E00427F400075
:1001F00072494949462141494D331814127F10274D
:10020000454545393C4A494931412111090736499B
:10021000494936464949291E00001400000040346F
:100220000000000814224114141414140041221474
:100230000802015909063E415D594E7C1211127C9B
:100240007F494949363E414141227F4141413E7FFC
:10025000494949417F090909013E414151737F08DC
:1002600008087F00417F41002040413F017F081482
:1002700022417F404040407F021C027F7F040810E3
:100280007F3E4141413E7F090909063E4151215EC1
:100290007F09192946264949493203017F01033F55
:1002A0004040403F1F2040201F3F4038403F6314E4
:1002B00008146303047804036159494D43007F41E6
:1002C00041410204081020004141417F0402010223
:1002D0000440404040400003070800205454784048
:1002E0007F284444383844444428384444287F38DC
:1002F0005454541800087E090218A4A49C787F085E
:1003000004047800447D40002040403D007F1028D8
:10031000440000417F40007C047804787C08040499
:10032000783844444438FC1824241818242418FC31
:100330007C08040408485454542404043F44243CD6
:100340004040207C1C2040201C3C4030403C442845
:100350001028444C9090907C4464544C44000836DF
:10036000410000007700000041360800020102044D
:10037000023C2623263C1EA1A161123A4040207A6D
:1003800038545455592155557941225454784221B5
:100390005554784020545579400C1E5272123955EC
:1003A00055555939545454593955545458000045E9
:1003B0007C410002457D420001457C407D121112C6
:1003C0007DF0282528F07C545545002054547C5459
:1003D0007C0A097F4932494949323A4444443A3215
:1003E0004A4848303A4141217A3A42402078009DBB
:1003F000A0A07D3D4242423D3D4040403D3C24FF67
:100400002424487E4943662B2FFC2F2BFF0929F615
:1004100020C0887E090320545479410000447D4166
:100420003048484A32384040227A007A0A0A727DBF
:100430000D19317D2629292F2826292929263048DA
:100440004D4020380808080808080808382F10C848
:10045000ACBA2F102834FA00007B000008142A14CC
:100460002222142A14085500550055AA55AA55AA47
:10047000FF55FF55FF000000FF00101010FF001493
:100480001414FF001010FF00FF1010F010F01414EF
:1004900014FC001414F700FF0000FF00FF1414F414
:1004A00004FC141417101F10101F101F1414141F15
:1004B00000101010F0000000001F101010101F108E
:1004C000101010F010000000FF101010101010108D
:1004D0001010FF10000000FF140000FF00FF0000DC
:1004E0001F10170000FC04F414141710171414F450
:1004F00004F40000FF00F714141414141414F7008B
:10050000F7141414171410101F101F141414F414DB
:100510001010F010F000001F101F0000001F14004A
:100520000000FC140000F010F01010FF10FF141475
:1005300014FF141010101F00000000F010FFFFFF48
:10054000FFFFF0F0F0F0F0FFFFFF0000000000FF01
:10055000FF0F0F0F0F0F3844443844FC4A4A4A3407
:100560007E02020606027E027E026355494163381E
:1005700044443C04407E201E2006027E020299A5CF
:10058000E7A5991C2A492A1C4C7201724C304A4D2D
:100590004D303048784830BC625A463D3E49494962
:1005A000007E0101017E2A2A2A2A2A44445F44440B
:1005B00040514A444040444A51400000FF0103E09A
:1005C00080FF000008086B6B083612362436060FD1
:1005D000090F06000018180000001010003040FF3E
:1005E0000101001F01011E00191D1712003C3C3CB7
:1005F0003C0000000000000103070F1F3F7F008048
:10060000C0E0F0F8FCFEDB40A4A62EAF2000A1C89D
:10061000D300408DAED580A800006000000000002F
:10062000000000000000000000E0000000000000EA
:100630000000000000000001E000000000000000D9
:1006400000000000000001F00000000000000000B9
:10065000000000000003F0000000000000000000A7
:100660000000000007F00000000000000000000093
:1006700000000007F800000000000000000000007B
:1006800000000FF800000003C0007E000001E00041
:100690007F0FF800000003C000FE000001E000FF33
:1006A000EFF800000003C000FE000001E000FFFFC3
:1006B000F800000003C000F00000000F007FFE7F84
:1006C000C0000003C000F00000000F003FFE7FF8F4
:1006D0003FF1FBCFFCFEF3BC3DEFE01FFE7FFF7F51
:1006E000FBFFDFFEFEFFBC3DEFE01FC6FFFF7FFB11
:1006F000FFDFFEFEFFBC3DEFE00FE3C7FE787BC3EC
:10070000DE1EF0FFBC3DEF0007FF87FC787BC3DEF9
:100710001EF0F83C3DEF0001FFFFF0007BC3C01E60
:10072000F0F03C3DEF0001F37FE03FFBC3CFFEF074
:10073000F03C3DEF0003E33F807FFBC3DFFEF0F0C2
:100740003C3DEF0007E73C00787BC3DE1EF0F03C49
:100750003DEF0007FFBE00787BC3DE1EF0F03C3D9E
:10076000EF0007FFFE00787BC3DE1EF0F03C3DEF9C
:10077000000FFFFE007FFBFFDFFEF0F03FFDEFE02C
:100780000FFFFF007FFBFFDFFEF0F03FFDEFE00F0C
:10079000F9FF003E79F9CF9EF0F01F3DE7E01FF131
:1007A000FF0000000000000000000000001F80FFAC
:1007B000007FFFFFFFFFFFFFFFFFFFE01C007F0048
:1007C0007FFFFFFFFEB46D888D18E000001F007FE3
:1007D000FFFFFFFE95AD7DB577E000000F007FFFC6
:1007E000FFFFFEA5AD9D8D19E0000006007FFFFF15
:1007F000FFFEB5ADEDB57EE0000000000001800019
:100800000000000000000000038000000000000065
:1008100000000007C000000000000000000007C04A
:100820000000000000000000000FC00000000000F9
:10083000000000001FE00000000000000000001F9A
:10084000E00000000000000000003FE000000000A9
:1008500000000000003FF000000000000000000069
:100860007FF0000000000000001FF87FF000000093
:10087000000000003FFE7FF0000000000000003F8D
:10088000FF7FF0000000000000001FFFFBE0000001
:1008900000000000000FFFF9FFC000000000000092
:1008A0000FFFF9FFF800000000000007FFF1FFFF55
:1008B00000000000000003FC73FFFF800000000048
:1008C0000001FE3FFFFF80000000000000FF1E0F40
:1008D000FF000000000000007FFE1FFC0000000081
:1008E0000000003FFFFFF8000000000000000FDFE5
:1008F000FFE0000000000000001F19FFC000000022
:10090000000000003F3CFF00000000000000007EEF
:100910007CF800000000000000007FFE7C0000006A
:100920000000000000FFFFFC0000000000000000CD
:10093000FFFFFE0000000000000000FFFFFE0000BF
:10094000000000000001FFEFFE00000000000000BA
:1009500001FFCFFE0000000000000003FF07FE00C3
:1009600000000000000003FC07FE00000000000083
:100970000003F003FE00000000000000018000FE04
:10098000000000000000000000007E0000000000E9
:1009900000000000003E0000000000000000000019
:1009A0000C000000000000078000FC000003C000F5
:1009B0000000078001FC000003C000000007800168
:1009C000FC000003C0000000078001E00000001EE2
:1009D000000000078001E00000001E007FE3F79F99
:1009E000F9FDE7787BDFC0FFF7FFBFFDFDFF787BF8
:1009F000DFC0FFF7FFBFFDFDFF787BDFC0F0F787AB
:100A0000BC3DE1FF787BDE00F0F787BC3DE1F0788C
:100A10007BDE0000F787803DE1E0787BDE007FF73A
:100A2000879FFDE1E0787BDE00FFF787BFFDE1E017
:100A3000787BDE00F0F787BC3DE1E0787BDE00F0FC
:100A4000F787BC3DE1E0787BDE00F0F787BC3DE155
:100A5000E0787BDE00FFF7FFBFFDE1E07FFBDFC05A
:100A6000FFF7FFBFFDE1E07FFBDFC07CF3F39F3DBD
:100A7000E1E03E7BCFC0000000000000000000006D
:100A800000FFFFFFFFFFFFFFFFFFFFC0FFFFFFFFB4
:100A9000FD68DB111A31C0FFFFFFFFFD2B5AFB6A17
:100AA000EFC0FFFFFFFFFD4B5B3B1A33C0FFFFFFB3
:100AB000FFFD6B5BDB6AFDC052455632205052454C
:100AC0005000563A00001FFC0000007FFF000001AC
:100AD000FFFFC00003FC1FE00007E003F0000F80F1
:100AE00000F8001F00007C001E00003C003C0000DD
:100AF0001E003C00001E00780C180F00781E3C0FF2
:100B000000701E3C0700F01E3C0780F01E3C078072
:100B1000F01E3C0780F01E3C0780F00C1807800098
:100B2000000000000000000000040C1810000F1E60
:100B30003C78000F1E3C78001E0C183C001E000084
:100B40003C003C00001E003C00001E007800000F2E
:100B5000007800000F00F000000780F00000078020
:100B6000F0000007807800000F007C00001F003EAE
:100B700000003E003FFFFFFE001FFFFFFC0007FFDD
:100B8000FFF00001FFFFC00000000000240027006C
:100B90002A0000000000250028002B0000000000B3
:100BA00023002600290004040404040404040202AF
:100BB00002020202030303030303010204081020DC
:100BC00040800102040810200102040810200000E7
:100BD00000080002010000030407000000000000FC
:100BE00000002200FF210000681E132511241FBEF3
:100BF000CFEFD8E0DEBFCDBF11E0A0E0B1E0E4E789
:100C0000FFE402C005900D92A03DB107D9F723E0A3
:100C1000A0EDB1E001C01D92A935B207E1F715E0E2
:100C2000C5EFD5E004C02197FE010E947626C43F9F
:100C3000D107C9F70E94F61E0C94AD270C94000052
:100C40000895833081F028F4813099F08230A9F042
:100C500008958730A9F08830C9F08430B1F48091CC
:100C600080008F7D03C0809180008F77809380000B
:100C7000089584B58F7784BD089584B58F7DFBCFAB
:100C80008091B0008F778093B00008958091B0007C
:100C90008F7DF9CFCF93DF93282F30E0F901E25316
:100CA000F44F8491F901E654F44FD491F901EA55D7
:100CB000F44FC491CC23A1F081110E942106EC2FA6
:100CC000F0E0EE0FFF1FE456F44FA591B491EC91C4
:100CD000ED2381E090E009F480E0DF91CF91089569
:100CE00080E090E0FACF1F93CF93DF93282F30E07E
:100CF000F901E253F44F8491F901E654F44FD49191
:100D0000F901EA55F44FC491CC23A9F0162F8111B3
:100D10000E942106EC2FF0E0EE0FFF1FEE56F44F7D
:100D2000A591B4918FB7F894EC91111108C0D095AA
:100D3000DE23DC938FBFDF91CF911F910895DE2BCF
:100D4000F8CFCF93DF9390E0FC01E654F44F249169
:100D50008A55944FFC0184918823D1F090E0880F4C
:100D6000991FFC01E857F44FA591B491FC01EE5690
:100D7000F44FC591D491623071F49FB7F8943C91CF
:100D8000822F809583238C93E8812E2B28839FBF0D
:100D9000DF91CF9108958FB7F894EC912E2B2C937F
:100DA0008FBFF6CF8E50806480937C0080917A0054
:100DB000806480937A0080917A0086FDFCCF8091D8
:100DC00078009091790008953FB7F8948091E602F9
:100DD0009091E702A091E802B091E90226B5A89BA4
:100DE00005C02F3F19F00196A11DB11D3FBFBA2FBD
:100DF000A92F982F8827BC01CD01620F711D811D7D
:100E0000911D42E0660F771F881F991F4A95D1F701
:100E100008958F929F92AF92BF92CF92DF92EF92FE
:100E2000FF924B015C010E94E4066B017C010E9471
:100E3000E4066C197D098E099F09683E734081059F
:100E40009105A8F321E0821A9108A108B10888EE63
:100E5000C80E83E0D81EE11CF11C81149104A1048A
:100E6000B10429F7FF90EF90DF90CF90BF90AF9043
:100E70009F908F9008952FB7F8946091E20270913F
:100E8000E3028091E4029091E5022FBF0895089556
:100E900008950895AF92BF92CF92DF92EF92FF92A2
:100EA0000F931F93CF93DF936C017B018B01040F92
:100EB000151FEB015E01AE18BF08C017D10759F02E
:100EC0006991D601ED91FC910190F081E02DC60170
:100ED0000995892B79F7C501DF91CF911F910F916A
:100EE000FF90EF90DF90CF90BF90AF900895EF927A
:100EF000FF920F931F93CF93DF93EC01EC80FD8063
:100F00006E157F050CF070C057FF04C0240F351F0D
:100F100050E040E08E819F81FA01E20FF31F8E17AF
:100F20009F071CF49C01241B350B121613060CF0B2
:100F30005BC0922F842F8695869586958E9DD001D5
:100F40008F9DB00D11246A0F7B1FAF8DB8A1A60F26
:100F5000B71F477049F188E0841B482F682F70E065
:100F6000FB01E250FA4FE491281708F063C0621BBE
:100F700071092FEF30E002C0359527956A95E2F7A9
:100F8000E2230130110539F0B0F10230110561F5AD
:100F90008C91E82702C08C91E82BEC93941720F1F8
:100FA0002C813D81A20FB31FE92FE41BE83078F0BC
:100FB0000230110521F58E2F9C9190959C932C81E8
:100FC0003D81A20FB31F88508830B0F7E770EE2341
:100FD00059F0F0E0EA50FA4FE49101301105F9F0D0
:100FE00010F10230110519F1DF91CF911F910F918E
:100FF000FF90EF900895E0958C91E823CECF81E0AB
:101000000115110509F480E081959E2F8C932C81A8
:101010003D81A20FB31F98509830C0F7D7CF8C9165
:10102000E82BEC93E1CFE0958C91E823FACF8C91FB
:10103000E827F7CF0130110509F4ADCFE0F2023017
:10104000110509F4A5CFAE0DBF1DAECF0F931F93B1
:10105000CF93DF9377FF04C0260F371F70E060E067
:10106000DC011496CD91DC91FB01E20FF31FCE174A
:10107000DF071CF49E01261B370B121613064CF5D6
:10108000FA0157FD3796A3E0F595E795AA95E1F7A4
:10109000EC9FD001ED9FB00DFC9FB00D11246A0FA5
:1010A0007B1FDC015F96ED91FC91E60FF71F477007
:1010B000552781E090E001C0880F4A95EAF7482F54
:1010C0000130110559F0A8F02E0F3F1F0230110515
:1010D000E1F0DF91CF911F910F9108952E0F3F1FE7
:1010E000E217F307B1F38191DF011197842B8C9301
:1010F000F7CF80952E0F3F1FE217F30751F3919121
:10110000DF01119798239C93F7CFE217F30709F3B8
:101110008191DF01119784278C93F7CF0F931F9351
:10112000FA01DC0156964C9156974230E9F0433073
:10113000A1F1413061F514964D915C91DA01AE1B3D
:10114000BF0BFD01E21BF30B77FD0BC0DC01169614
:101150004D915C916417750724F4AB01BF010E94A7
:1011600026081F910F91089514964D915C91DA0114
:10117000A61BB70BBD0161507109DC0116964D919C
:101180005C91DA01AE1BBF0BFD01E21BF30B77FD97
:10119000E8CFAF010E947707E4CF16964D915C919E
:1011A000DA01A61BB70BBD0161507109CDCF0F93BA
:1011B0001F93FA01DC0156964C9156974230A9F0E4
:1011C000433091F1413019F514964D915C91DA015B
:1011D000AE1BBF0BFD013197F7FD04C0AB01BF0192
:1011E0000E9477071F910F91089514964D915C917D
:1011F000DA01A61BB70BBD01DC0116964D915C917F
:10120000DA01AE1BBF0BFD013197621B730BF7FDBB
:10121000E9CFDC0116964D915C91E417F50714F7C0
:10122000AF010E942608DECF16964D915C91DA013F
:10123000A61BB70BBD01621B730BCECFFC0177FD64
:1012400064C080859185681779070CF05EC057FDF2
:101250005CC082859385481759070CF056C0868973
:101260008230B1F0833029F1813041F4848195815D
:10127000841B950BAB01BC01615071092130310514
:1012800009F108F443C02230310509F463C0089520
:1012900084819581DC01A61BB70BBD0161507109EA
:1012A00086819781DC01A41BB50BAD01415051092A
:1012B000E5CF86819781861B970BBA01AC0141501F
:1012C0005109DCCFCA0157FD0796A3E09595879594
:1012D000AA95E1F7A481B5818A9F90018B9F300D7B
:1012E0009A9F300D1124620F731F078CF0A1E02D1F
:1012F000E60FF71F4770552721E030E001C0220FAD
:101300004A95EAF78081822B80830895CA0157FDB0
:10131000079633E0959587953A95E1F7A481B581D5
:101320008A9F90018B9F300D9A9F300D1124620F80
:10133000731F078CF0A1E02DE60FF71F47705527AC
:1013400081E090E001C0880F4A95EAF7809590818E
:101350008923DACFCA0157FD079623E09595879533
:101360002A95E1F7A481B5818A9F90018B9F300D6A
:101370009A9F300D1124620F731F078CF0A1E02D8E
:10138000E60FF71F4770552721E030E001C0220F1C
:101390004A95EAF780818227B7CF08958EBD000075
:1013A0000DB407FEFDCF8EB508958CBD9DBD08958B
:1013B0000895FC016370668B848195812681378155
:1013C000613039F0633029F0918780873387228735
:1013D0000895318720879387828708952F923F92BF
:1013E0004F925F926F927F928F929F92AF92BF9235
:1013F000CF92DF92EF92FF920F931F93CF93DF93E1
:10140000CDB7DEB76A970FB6F894DEBF0FBECDBF7B
:101410009A8F898F7A8369834A01D22E18870F8326
:101420003701BC2CDC0159962D913C915A9721151E
:10143000310509F015C118968D919C91199768177F
:1014400079070CF0D7C11A968D919C9148175907CE
:101450000CF0D0C14C2C512CB6E0CB9E600D711D10
:1014600011247C876B87161617060CF0C3C1EA2D72
:10147000F0E0FA87E98793E0EE0FFF1F9A95E1F716
:10148000F88BEF87CF01840F951F181619060CF003
:10149000B1C1A98DBA8D58968C91811104C0BFEA53
:1014A000BD1508F4D394A98DBA8DED91FC911197D7
:1014B0000284F385E02DCD010995B5E0DB9EC001E6
:1014C0001124E981FA81FC83EB83312C212C9C01CE
:1014D0002A503F4F388F2F8B4A2D50E05E8B4D8B1B
:1014E000EF89F88DE20DF31D44919E828D82D12CFF
:1014F000C12C69817A81620D731D7A8B698B842F6F
:1015000090E09C8B8B8BE98DFA8DA081B18140FF9F
:1015100082C0F1E0BF126FC0AF126DC01C96ED919A
:10152000FC912F813885A4014C0D5D1D69897A8954
:10153000898D9A8D0995EB89FC89F595E7954E2F54
:101540005FEFC51AD50A6D817E818D899E89680FEE
:10155000791F7E836D8398E0C916D10481F6AFEFC1
:101560002A1A3A0AEB81FC81E40DF51DFC83EB831A
:10157000F5E02F16310409F0B3CF2F8138852615F9
:101580003705B9F0A98DBA8DED91FC91B1E0BB1290
:1015900057C0AB1255C069817A816B5F7F4F00885D
:1015A000F189E02D830128E030E0A401898D9A8D36
:1015B0000995A98DBA8DED91FC9111970688F7894F
:1015C000E02DCD016A960FB6F894DEBF0FBECDBFF9
:1015D000DF91CF911F910F91FF90EF90DF90CF900F
:1015E000BF90AF909F908F907F906F905F904F9043
:1015F0003F902F9009941E96ED91FC91EF80F88416
:1016000009851A8592014D815E816B817C81898D6E
:101610009A8D099590CF2F8138852615370509F4C5
:101620008ACF31E0B31207C0A31205C01C96ED911A
:10163000FC91930178CF1E96ED91FC917301E0CF60
:101640006B857C85641975090684F785E02D730127
:101650000F8518899201A401898D9A8D0995A9CFCA
:10166000F90134969491329745915491D91AB7E083
:10167000DB9E400D511D1124F901259134913C8BC5
:101680002B8BFA0125903490FA01329674903196A2
:101690003491398B329664903196449041E04C15E8
:1016A00018F04A1508F07FC0662D062C000C770B49
:1016B0007C836B83842D042C000C990B9E838D837B
:1016C000A98DBA8DED91FC9111970284F385E02DDF
:1016D000CD010995512CD12CC12CEA2DF0E0FA87CF
:1016E000E9872B2D30E03C872B87A401440D511D49
:1016F00047FC5A95588F4F8B69817A81660D711D11
:1017000067FC7A957E876D877989C71608F051CF77
:101710002C2D30E04D815E81420F531FA985BA8583
:101720004A9FC0014B9F900D5A9F900D1124FC01C0
:10173000E80DF91DF88BEF87852D612C4F89588DA9
:10174000420F531F5E8B4D8B671408F050C044242A
:101750004394480E877041F4C1010196EB89FC89DE
:10176000E20DF31DD4901C01D7FE19C0A98DBA8DCE
:10177000ED91FC91662D70E0B1E0BB1219C0AB1287
:1017800017C02D853E85620F731F0484F585E02DFB
:101790002F8138854D895E89898D9A8D0995DD0C5B
:1017A0006394842DD1CF1E821D821C821B8288CF20
:1017B0004B815C81640F751FAB85BC856A9FC0013E
:1017C0006B9F900D7A9F900D112469817A81680F2B
:1017D000791F0684F785E02DEF80F88409851A8546
:1017E0009D014F855889898D9A8D0995D8CF570CC1
:1017F000C3948ACF6A960FB6F894DEBF0FBECDBFF2
:10180000DF91CF911F910F91FF90EF90DF90CF90DC
:10181000BF90AF909F908F907F906F905F904F9010
:101820003F902F9008958F929F92AF92CF92EF9218
:10183000FF920F931F93CF93DF93EC01262F898D97
:101840009A8D009709F051C06A30D1F41D861C862C
:101850008D8948E0849F900111248E859F85820F99
:10186000931F9F878E8781E090E0DF91CF911F913A
:101870000F91FF90EF90CF90AF909F908F90089531
:101880006D3089F3CC88AD888F898823C1F08C8531
:101890009D8536E0C39E800D911D11244885598594
:1018A0004817590764F44E855F851D861C8638E00D
:1018B000A39EC0011124840F951F9F878E87EA88FD
:1018C000FB88088919894E855F856C857D85CE01E9
:1018D0000E94EE092C898C859D8546E0249F800D11
:1018E000911D11249D878C87BECF6A3069F41D86B7
:1018F0001C86FC013896E4912D898E859F85E29F98
:10190000800D911D1124ADCF6D3009F4ACCFFC01D9
:1019100034963491631708F4A6CF3296E491E61713
:1019200008F4A1CFFC01329685909490462F431B7A
:10193000342F47E0349F800C911C1124F40132961F
:1019400034913196E4913323A9F1EE2399F1CC88B7
:10195000F4013596E491AD884F89442301F10E2EB0
:10196000000CFF0BE30FF11DCE9EA001CF9E500D8A
:1019700011246C857D85460F571F6885798564170E
:1019800075076CF44E855F851D861C86FC013896B4
:10199000E491AE9E400D511D11245F874E87EA8869
:1019A000FB88088919894E855F856C857D85CE0108
:1019B0000E94EE09F4013496E4912C898C859D8572
:1019C000E29F800D911D11248DCF0F931F93CF9314
:1019D000DF938C01D0E0C0E0F801EC0FFD1F6491B3
:1019E000662341F085E193E00E94130C892B11F0EE
:1019F0002196F2CFCE01DF91CF911F910F910895E3
:101A00006F927F928F929F92AF92BF92CF92DF920E
:101A1000EF92FF920F931F93CF93DF93EC016B0133
:101A20005A0139014801E881F9810284F385E02DEA
:101A30000995E881F9810288F389E02D87019301F6
:101A4000A501B601CE010995A501480D591D4150CA
:101A50005109E881F9810288F389E02D9301B601EB
:101A6000CE010995E881F9810088F189E02D940182
:101A7000A501B601CE010995C60CD71CB60161506F
:101A80007109E881F9810088F189E02D9401A501AF
:101A9000CE010995E881F9810688F789E02DCE010C
:101AA000DF91CF911F910F91FF90EF90DF90CF903A
:101AB000BF90AF909F908F907F906F9009946F929E
:101AC0007F928F929F92AF92BF92CF92DF92EF92CE
:101AD000FF920F931F93CF93DF935C01EB016A0199
:101AE000490138018701DC01ED91FC916217730710
:101AF00019F5641675062CF0962D872D3A01C92E1E
:101B0000D82E9601261937092F5F3F4F048CF58D8B
:101B1000E02DA301BE01C5010995DF91CF911F9171
:101B20000F91FF90EF90DF90CF90BF90AF909F907C
:101B30008F907F906F9008954615570591F4261762
:101B4000370724F0892D4B01C22FD82F9E01281969
:101B500039092F5F3F4F068CF78DE02DA601B401A8
:101B6000DACF0284F385E02D0995D501ED91FC9142
:101B70000488F589E02D83019401A601BE01C50109
:101B80000995D501ED91FC910688F789E02DC501F5
:101B9000DF91CF911F910F91FF90EF90DF90CF9049
:101BA000BF90AF909F908F907F906F900994EF922D
:101BB000FF920F931F93DC011A960D911C911B97B6
:101BC00018962D913C911997ED91FC9100A0F1A1EF
:101BD000E02D7B0150E040E070E060E009951F914E
:101BE0000F91FF90EF9008954F925F926F927F92C6
:101BF0008F929F92AF92BF92CF92DF92EF92FF921D
:101C00000F931F93CF93DF936C012B015A0139017E
:101C10004801DC01ED91FC910284F385E02D0995EA
:101C2000E201640C751CD601ED91FC91C615D70537
:101C30005CF40088F189E02D87019401A501BE01C3
:101C4000C60109952196EFCF0688F789E02DC601D8
:101C5000DF91CF911F910F91FF90EF90DF90CF9088
:101C6000BF90AF909F908F907F906F905F904F90BC
:101C700009948F929F92AF92BF92CF92DF92EF9290
:101C8000FF920F931F93CF93DF93EC015B014A0107
:101C90006901E881F9810284F385E02D09959501B8
:101CA0002C0D3D1D21503109E881F9810488F58909
:101CB000E02D78018401A401B501CE010995E881E8
:101CC000F9810688F789E02DCE01DF91CF911F9130
:101CD0000F91FF90EF90DF90CF90BF90AF909F90CB
:101CE0008F9009948F929F92AF92BF92CF92DF9282
:101CF000EF92FF920F931F93CF93DF93EC015B0161
:101D00004A0169017801E881F9810284F385E02DB7
:101D10000995C80CD91C860101501109E881F98187
:101D20000488F589E02D9501A401B501CE0109953E
:101D3000E881F9810688F789E02DCE01DF91CF9106
:101D40001F910F91FF90EF90DF90CF90BF90AF90D9
:101D50009F908F900994EF92FF920F931F93DC0155
:101D6000ED91FC9100A0F1A1E02D09951F910F913B
:101D7000FF90EF9008950F931F93DC01ED91FC917C
:101D8000068CF78DE02D09951F910F9108950F9303
:101D90001F93DC01ED91FC91048CF58DE02D0995EC
:101DA0001F910F910895DC01ED91FC910084F18564
:101DB000E02D09943F924F925F926F927F928F92A3
:101DC0009F92AF92BF92CF92DF92EF92FF920F93CA
:101DD0001F93CF93DF9300D000D0CDB7DEB75C0167
:101DE0003B016A014901280187E0480E511C93E03C
:101DF000559447949A95E1F7CA018E0D9F1D9A83D9
:101E00008983F12CE12C312C1C821B828B819C81DB
:101E100087709927330C892B61F4EB81FC8183E077
:101E2000F595E7958A95E1F7EE0DFF1DE80DF91D93
:101E3000349037FE0AC021E030E0A6016B817C813E
:101E4000660D771DC5010E94D30E8B819C81019682
:101E50009C838B8308171907C9F69FEFC91AD90A03
:101E6000E40CF51C89819A81C816D90669F60F9091
:101E70000F900F900F90DF91CF911F910F91FF90D6
:101E8000EF90DF90CF90BF90AF909F908F907F901A
:101E90006F905F904F903F9008952F923F924F9296
:101EA0005F926F927F928F929F92AF92BF92CF92EA
:101EB000DF92EF92FF920F931F93CF93DF9300D0A7
:101EC00000D000D0CDB7DEB73C016A013E832D8340
:101ED000FC82EB825801A41AB50AB7FE03C0B19484
:101EE000A194B1088D809E80861A970A97FE03C040
:101EF0009194819491088A149B045CF0902F812F17
:101F00000D811E819D838E839C2D8D2D6B01692FEC
:101F1000782F0C151D055CF09D818E817E836D836D
:101F2000692F782F902F812F8601C92ED82E160168
:101F3000201A310A2B012D813E81421A530A57FE85
:101F400003C0519441945108710137FE03C03FEF23
:101F5000E31AF30AF594E7948D819E81861797071B
:101F60005CF5A1E0B0E0BA83A983C016D1064CF1BC
:101F7000D301ED91FC910484F585E02D2B813C810A
:101F8000A8016D817E818A149B041CF04D815E81C5
:101F9000B801C3010995E418F508F7FE0AC02D81C0
:101FA0003E8189819A81280F391F3E832D83E20C5F
:101FB000F31C0F5F1F4FD9CF2FEF3FEF3A832983D9
:101FC000D4CF26960FB6F894DEBF0FBECDBFDF91FB
:101FD000CF911F910F91FF90EF90DF90CF90BF9026
:101FE000AF909F908F907F906F905F904F903F90B9
:101FF0002F900895089520915F02260F3327331FF5
:1020000021323105ECF420918302FC0190E080E064
:10201000243069F082E00895A0915F022191AC0123
:10202000415C5D4FA40FB52FB11D2C93019686170F
:1020300098F380915F02680F60935F0280E00895DB
:1020400081E008951092830281E0809385021092CE
:10205000840261E082E10E94730661E083E10E94F4
:102060007306E9EBF0E080818E7F808380818D7F35
:10207000808388E48093B80085E48093BC00089551
:10208000CF93DF9391E090933E028823B9F0C09103
:10209000B800D091BA008091BC008A7B8093BC00CC
:1020A00060E082E10E94730660E083E10E947306B3
:1020B0000E942210D093BA00C093B800DF91CF9154
:1020C0000895E091AF028091AE02E81730F4F0E09D
:1020D000E75EFD4F808190E008958FEF9FEF0895B8
:1020E0009091AF028091AE022FEF3FEF981748F426
:1020F000E92FF0E0E75EFD4F208130E09F5F909395
:10210000AF02C90108958091AE029091AF02891B80
:10211000990B0895CF92DF92EF92FF920F931F9346
:10212000CF93DF937C01CB018A012091ED02222322
:1021300089F0EB016B01C40ED51ECC15DD0569F0ED
:102140006991D701ED91FC910190F081E02DC701DB
:102150000995F3CF642F0E94FB0FC801DF91CF9147
:102160001F910F91FF90EF90DF90CF900895CF9344
:10217000DF931F92CDB7DEB769832091ED02222352
:10218000F9F02091EA02203258F021E030E0FC0121
:102190003383228390E080E00F90DF91CF91089508
:1021A0008091EB02E82FF0E0E750FE4F9981908399
:1021B0008F5F8093EB028093EA0281E090E0ECCFA6
:1021C00061E0CE0101960E94FB0FF7CFCF92DF9224
:1021D000EF92FF920F931F93CF93DF93D091EA0278
:1021E00081E0D13208F09CC0C091EC020E94E4066C
:1021F0006B017C018091830281116CC082E080932D
:10220000830281E0809385028FEF80938202109297
:10221000A702D093A602A9EFB1E0E6E8F2E080E0E1
:10222000D8138DC01092A8028091A802CC0FC82BA1
:10223000C093A80280918402813009F084C010927A
:1022400084020E94E4066B017C018091A8028093C5
:10225000BB0080913A0290913B02A0913C02B09168
:102260003D02892B8A2B8B2BA1F00E94E406009162
:102270003A0210913B0220913C0230913D026C19D0
:102280007D098E099F09061717072807390708F4E3
:1022900042C08091BC0083FDD8CF85EC8093BC0008
:1022A0000E94E4066B017C0180918302823009F474
:1022B0004CC0809182028F3F09F469C080918202F4
:1022C000803209F466C080918202803309F463C0D1
:1022D00084E026C080913A0290913B02A0913C029A
:1022E000B0913D02892B8A2B8B2B09F483CF0E945E
:1022F000E40600913A0210913B0220913C02309199
:102300003D026C197D098E099F09061717072807DA
:10231000390708F06FCF809139020E94401085E0A4
:102320001092EB021092EA021092ED02DF91CF912F
:102330001F910F91FF90EF90DF90CF9008959D91A6
:1023400091938F5F6DCF85EEA9CF80913A029091E6
:102350003B02A0913C02B0913D02892B8A2B8B2B32
:1023600009F4A2CF0E94E40600913A0210913B02C8
:1023700020913C0230913D026C197D098E099F0924
:10238000061717072807390708F08ECFC4CF80E05B
:10239000C7CF82E0C5CF83E0C3CFEF92FF920F9308
:1023A0001F93CF93DF937C01C62F809132039091CE
:1023B0003303009709F459C02091360331E030937C
:1023C000ED022093EC021092EB021092EA02DC0183
:1023D000ED91FC910190F081E02D60E0099587017D
:1023E000EE24E394F12CD1E0C1508091320390911E
:1023F0003303CF3F91F1B0E2EB16F104D8F00E9425
:10240000E610809132039091330320913603D093EC
:10241000ED022093EC021092EB021092EA02DC0132
:10242000ED91FC910190F081E02D60E00995EE24A2
:10243000E394F12C8091320390913303F80164917D
:10244000DC01ED91FC910190F081E02D0995BFEF49
:10245000EB1AFB0A0F5F1F4FC7CFDF91CF911F9180
:102460000F91FF90EF900C94E610E0914203F091F1
:10247000430390818091480380958923808387015D
:10248000C15008F438C0F801849120913003309194
:102490003103232B29F00E94CE090F5F1F4FF0CF8D
:1024A00028E030E040E8E0913E03F0913F03909156
:1024B0004603582F5423D9F05081952B9083E091F7
:1024C0004003F0914103908150914703952B9083F5
:1024D000E0914003F0914103508190914703909522
:1024E00095239083469521503109E9F6D6CF508146
:1024F00090959523E3CFDF91CF911F910F91FF909E
:10250000EF9008951F93CF93DF93EC018D8D9E8DF7
:10251000009721F1162F29A131E03093ED0220938D
:10252000EC021092EB021092EA02DC01ED91FC91B8
:102530000190F081E02D60E009958D8D9E8DDC018C
:10254000ED91FC910190F081E02D612F09958D8D29
:102550009E8DDF91CF911F910C94E610ADA5BEA585
:102560009C918BA9809589238C938B8D9C8D892B35
:1025700031F0862FDF91CF911F910C94CE0928E086
:1025800030E080E8A9A5BAA599A9462F4823C1F053
:102590004C91942B9C93ABA5BCA59C914AA9942BE0
:1025A0009C93ABA5BCA54C919AA9909594239C9320
:1025B00086952150310931F7DF91CF911F91089510
:1025C0004C9190959423E6CFDF92EF92FF920F9378
:1025D0001F93CF93DF938091320390913303892B24
:1025E00009F498C020914A0330914B0340914C0369
:1025F00050914D0360E074E284EF90E00E940E265B
:10260000205131094109510956954795379527952C
:102610002093B80065E082EE9BE00E94CD116091AE
:102620001903615085E193E00E94821220911B03FF
:1026300030911C03C901079697FD079633E09595E5
:1026400087953A95E1F72091190330911A03829FFB
:102650008001839F100D929F100D1124C0913403AF
:10266000D091350380913203909133030C0F1D1FDD
:10267000009709F48FC02091360331E03093ED02CA
:102680002093EC021092EB021092EA02DC01ED9131
:10269000FC910190F081E02D60E40995EE24E39433
:1026A000F12CDD24D39480913203909133030C17E5
:1026B0001D0709F446C0B0E2EB16F104D8F00E9401
:1026C000E610809132039091330320913603D0922B
:1026D000ED022093EC021092EB021092EA02DC0170
:1026E000ED91FC910190F081E02D60E40995EE24DC
:1026F000E394F12C80913203909133036991DC01D2
:10270000ED91FC910190F081E02D0995BFEFEB1A5E
:10271000FB0AC9CF8091300390913103892B31F0AE
:1027200080915303909154030E94D509E091440392
:10273000F09145039081809149038095892380839E
:1027400069CF0E94E6108091320390913303892B68
:1027500009F461C020914E0330914F034091500322
:102760005091510360E074E284EF90E00E940E26E5
:1027700020513109410951095695479537952795BB
:102780002093B800DF91CF911F910F91FF90EF90B0
:10279000DF900895E0914203F0914303808190918E
:1027A0004803892B80830C171D0769F289912091BA
:1027B000300330913103232B19F00E94CE09F3CF5F
:1027C00028E030E040E8E0913E03F0913F03909133
:1027D0004603582F5423D9F05081952B9083E091D4
:1027E0004003F0914103908150914703952B9083D2
:1027F000E0914003F09141035081909147039095FF
:1028000095239083469521503109E9F6CCCF50812C
:1028100090959523E3CFE0914403F09145038081A7
:1028200090914903892B8083ADCF1F93CF93DF9382
:10283000EC01162F8D8D9E8D892BB1F12DA93EA90E
:102840004FA958AD60E074E284EF90E00E940E263C
:1028500020513109410951095695479537952795DA
:102860002093B80066EA111167EACE010E94821235
:102870008D8D9E8D892B41F129AD3AAD4BAD5CAD6F
:1028800060E074E284EF90E00E940E26205131094E
:102890004109510956954795379527952093B800DA
:1028A000DF91CF911F9108958B8D9C8D892B21F005
:1028B0008EAD9FAD0E94D509EFA5F8A990818CA996
:1028C000809589238083CECFEFA5F8A980819CA92C
:1028D000892B8083E5CF90E080E008950F931F93CC
:1028E000CF93DF93CDEED1E00EE611E0199219926D
:1028F000F80180810E5F1F4F60E00E947306F1E0D7
:10290000C93FDF0799F71092EC011092EB0110928A
:10291000EA011092E901DF91CF911F910F91089583
:10292000CF92DF92EF92FF92C090E501D090E60146
:10293000E090E701F090E801C092E101D092E2015D
:10294000E092E301F092E4010E943B076093E5010D
:102950007093E6018093E7019093E8012091DC02F7
:10296000213009F042C06C197D098E099F096E372C
:10297000710581059105C0F01092EE011092ED01F4
:102980001092F0011092EF011092F2011092F101F9
:102990001092F4011092F3011092F6011092F501D9
:1029A0001092F8011092F7018091CE02811103C0BC
:1029B00081E08093CE021092EA011092E9018091A9
:1029C000EB019091EC018731910550F401969093C1
:1029D000EC018093EB01FF90EF90DF90CF90089592
:1029E0001092EC011092EB01F6CF223051F52091BC
:1029F000CE02211103C021E02093CE026C197D0983
:102A00008E099F09693B7B408105910520F00E945A
:102A10006E141092D2011092EA011092E901109204
:102A2000EC011092EB018091D201811104C081E090
:102A30008093D201D0CF813071F60E946E1482E073
:102A4000F7CF233041F62091CE02211103C021E0BF
:102A50002093CE026C197D098E099F096F3E72404A
:102A60008105910540F00E946E141092D2011092DF
:102A7000D1011092D0018091D0019091D1010097A5
:102A800099F41092EC011092EB011092EA0110926D
:102A9000E90101969093D1018093D0018091D201F8
:102AA000843050F48F5FC4CF8330910590F310923F
:102AB000D1011092D001F2CF843009F08CCF0E9466
:102AC0006E1485E0B5CF0F931F938091DC028111C6
:102AD0003BC02091D0022223A1F18AE0289F9001DF
:102AE00011248091CF02A091BF02B091C00288232F
:102AF00021F0A091BD02B091BE020E9453262FEF9B
:102B000033E040E050E00E94DC258091400190914C
:102B10004101280F391F48E1429FC001439F900D9A
:102B200011249C0150E040E060E67AEE80E090E005
:102B30000E94DC253093E0012093DF011F910F916B
:102B4000089530E020E0E1CF8230D9F46091E501D2
:102B50007091E6018091E7019091E8010091E10117
:102B60001091E2012091E3013091E401601B710BAF
:102B7000820B930B28E130E040E050E00E940E26EB
:102B8000D9CF8330D9F66091E5017091E60180914B
:102B9000E7019091E8010091E1011091E20120919B
:102BA000E3013091E401601B710B820B930B26E073
:102BB00030E040E050E0E2CF2F923F924F925F92A0
:102BC0006F927F928F929F92AF92BF92CF92DF923D
:102BD000EF92FF920F931F93CF93DF937090BD02FC
:102BE0006090BE025090BF024090C0020AE011E027
:102BF00092ECE92E92E0F92E23EDC22E21E0D22EA6
:102C000088248A9433E0932EA12CB12C48E1242E01
:102C1000312CF80125813681C081D1812115310502
:102C2000A9F5CC0FDD1FC45BDE4F88819981F601C9
:102C300091838083619171916F0116161706B4F527
:102C4000F8E1F69FC001F79F900D11240197F7015D
:102C500091838083075F1F4FF2E0EF0EF11C21E0AC
:102C600000341207B1F6DF91CF911F910F91FF90C1
:102C7000EF90DF90CF90BF90AF909F908F907F901C
:102C80006F905F904F903F902F9008958481A72D73
:102C9000B62D811102C0A52DB42D0E945326A50189
:102CA00094010E94DC25C21BD30BBBCF71956195AB
:102CB0007109C1010E943F2661507109F7017183BA
:102CC0006083C8CFFC0101900020E9F73197AF0184
:102CD000481B590BBC0185E193E00C944A078F9285
:102CE0009F92AF92BF920F931F93CF93DF93CDB775
:102CF000DEB7A1970FB6F894DEBF0FBECDBF19A205
:102D0000423008F44AE08E010F5D1F4F842E912C53
:102D1000B12CA12CA50194010E940E26E62FB90129
:102D2000CA01EA30F4F4E05DD801EE938D01232B63
:102D3000242B252B79F790E080E0109719F0CD0136
:102D40000E946216A1960FB6F894DEBF0FBECDBFEB
:102D5000DF91CF911F910F91BF90AF909F908F9077
:102D60000895E95CE1CFCF92DF92EF92FF92CF938B
:102D7000DF936C01990FEE08FF08F7FE19C06DE2B2
:102D800085E193E00E94130CEC0166277727CB01C5
:102D90006C197D098E099F094AE00E946F168C0FFD
:102DA0009D1FDF91CF91FF90EF90DF90CF9008951E
:102DB0004AE0C701B601DF91CF91FF90EF90DF901D
:102DC000CF900C946F1688EC91E00C946216CF9320
:102DD000DF930E94E50CEC010E94E3168C0F9D1F0F
:102DE000DF91CF91089520911B0330911C03C901FD
:102DF000079697FD079623E0959587952A95E1F725
:102E00002091190330911A03829FA001839F500DD6
:102E1000929F500D112470E060E0809134039091F6
:102E200035030C94A627EF92FF920F931F93CF9335
:102E3000DF930E94F3160E943B076093DD027093BC
:102E4000DE028093DF029093E002EE24E394F12C03
:102E500002E010E020E830E050E040E070E060E0A8
:102E600085E193E00E94000D10922203109221034D
:102E700082E090E0909324038093230381E0809389
:102E8000290380932A038091D3029091D402109257
:102E9000260310922503892B09F043C1C1E0D0E03D
:102EA000D0932803C093270384EF90E00E94E50CA1
:102EB000D0932803C0932703D0932603C093250300
:102EC0008EEE90E00E94E50CC1E0D0E001E010E061
:102ED0008091D3029091D402109226031092250380
:102EE00010932803009327038C179D0709F022C134
:102EF0008BEC91E00E946216109328030093270345
:102F000010932603009325038BEC91E00E94621638
:102F1000CE010E94B3168BEC91E00E9462162196BE
:102F2000C730D105A9F61092260310922503C1E0FF
:102F3000D0E0D0932803C0932703EE24E394F12C30
:102F400008E010E024E130E042E050E06CE670E0A0
:102F500085E193E00E94F40D0E94E3160E94E316BF
:102F600002E010E020E830E04AE050E070E060E08D
:102F700085E193E00E94F40D84E090E090932203B9
:102F80008093210380E190E09093240380932303B6
:102F900083E08093290380932A03D0932803C0936E
:102FA0002703D0932603C09325032091D3023091A9
:102FB000D4022115310509F0FEC08091DC02811197
:102FC000C1C080914001909141018436910520F467
:102FD0008BEC91E00E94621660914001709141017A
:102FE00090E080E04AE00E946F160E94E31685E1BF
:102FF00090E0909322038093210388E290E09093E5
:1030000024038093230382E08093290380932A037F
:1030100085EE90E00E94E7160E94E316C1E0C0939F
:103020002903C0932A030E94E3168AE390E0909359
:1030300022038093210380E190E090932403809306
:103040002303C0932903C0932A032091D302309114
:10305000D4028091D5029091D602232B09F014C19D
:103060008130910509F0E8C01092260310922503E3
:10307000909328038093270384EC90E00E94E50C52
:103080008091DC02813009F0E2C08DEB90E00E947B
:10309000E7168091D5029091D602029709F0E4C01C
:1030A000109226031092250381E090E0909328036C
:1030B000809327038AE390E0909322038093210377
:1030C0008EE190E0909324038093230384EA90E0C0
:1030D0000E94E50C8091D002882309F4D0C0809131
:1030E000DC028111CCC081EA90E00E94E50C809165
:1030F000CF0290E001960E94B3168DEC91E00E9401
:1031000062168091D0022AE0829FC00111240E94A1
:10311000B316DF91CF911F910F91FF90EF900C9418
:10312000E41281E090E0909328038093270389EED6
:1031300090E0C8CE8BEC91E00E946216CE010E9416
:10314000B316EDCE8130C1F481EE90E00E94E71617
:1031500088E090E0909322038093210388E290E03E
:10316000909324038093230382E080932903809328
:103170002A038CED90E04ECF823069F428E030E0F5
:1031800030932203209321038093290380932A0301
:1031900087ED90E03FCF833071F488E090E090932A
:1031A00022038093210382E08093290380932A03E2
:1031B00082ED90E02FCF21503109C9E0C29FF0018C
:1031C000C39FF00D1124E65FFE4F0190F081E02DCA
:1031D000EE0FFF1FE45BFE4F80819181009729F481
:1031E0008EEC90E00E94E50C17CF181619060CF52E
:1031F0008CEC90E00E94E50C8091D3029091D40277
:103200000197C89FF001C99FF00D1124E65FFE4FA2
:103210000190F081E02DEE0FFF1FE45BFE4F8081F7
:10322000918197FF03C09195819591090E94B316F2
:10323000F3CE8AEC90E0DECF81E090E0909328031B
:1032400080932703909326038093250315CF823024
:1032500019F486EB90E01BCF833019F48FEA90E0ED
:1032600016CF8AEA90E013CF81E090E09093280394
:103270008093270390932603809325031BCF8CE92B
:1032800090E00E94E50C45CF8130910509F0D7C050
:10329000109226031092250390932803809327030E
:1032A00086E990E00E94E50C8091D3029091D402CF
:1032B000019729E0289FF001299FF00D1124E65F76
:1032C000FE4F628173818DE890E06115710539F0E0
:1032D00090E080E04AE00E946F1682E990E00E9450
:1032E000E50C8091D5029091D602029709F0B2C008
:1032F000109226031092250381E090E0909328031A
:10330000809327038AE390E0909322038093210324
:103310008EE190E0909324038093230387E890E06C
:103320000E94E50C8091D3029091D4020197C9E0EC
:10333000C89FF001C99FF00D1124E65FFE4F248164
:1033400085819681222309F490C0892B09F4BCC0A1
:1033500083E890E00E94E50C8091D3029091D40222
:103360000197C89FF001C99FF00D1124E65FFE4F41
:10337000858196811816190624F481E890E00E9450
:10338000E50C8091D3029091D402019729E0289F07
:10339000F001299FF00D1124E65FFE4F8581968193
:1033A0000E94B3168FE790E00E94E50C8091D50251
:1033B0009091D602039709F08AC0109226031092CA
:1033C000250381E090E090932803809327038AE30C
:1033D00090E090932203809321038CE290E09093FD
:1033E0002403809323038CE690E00E94E50C8091F7
:1033F000D3029091D402019729E0289FF001299FE0
:10340000F00D1124E65FFE4F6781708590E080E04B
:103410004AE00E946F168AE690E00E94E50CE09177
:10342000D302F091D402EE0FFF1FE054FD4F8081D4
:10343000918101960E94B31688E690E022CF81E048
:1034400090E0909328038093270390932603809322
:10345000250326CF81E090E09093280380932703F3
:1034600090932603809325034DCF892B69F18BE739
:1034700090E00E94E50C8091D3029091D4020197D4
:10348000C89FF001C99FF00D1124E65FFE4F8581B2
:1034900096811816190624F489E790E00E94E50C3D
:1034A0008091D3029091D402019729E0289FF001E6
:1034B000299FF00D1124E65FFE4F858196810E94C1
:1034C000B31687E790E070CF82E790E06DCF81E0A0
:1034D00090E0909328038093270390932603809392
:1034E000250375CFFF920F931F93CF93DF93EC01CA
:1034F000F62E08811981C8010E94C625F81621F010
:103500006F2DC8010E94CE25CE01DF91CF911F9172
:103510000F91FF900895EF92FF920F931F93CF9317
:10352000DF9300D0CDB7DEB71A82198260914001D7
:10353000CE0101960E94721A81E090E09A838983FD
:1035400060914101CE0101960E94721A82E090E0E2
:103550009A8389836091CF02CE0101960E94721AEC
:1035600083E090E09A8389836091D002CE01019636
:103570000E94721A84E090E09A8389836091DC0251
:10358000CE0101960E94721A8AE0E82E81E0F82EA0
:1035900005E010E01A830983F70161917F01CE01F4
:1035A00001960E94721A0F5F1F4F0B33110591F79E
:1035B0000F900F90DF91CF911F910F91FF90EF909F
:1035C0000895CF93DF93EB010E94C6258883CE0137
:1035D000DF91CF9108950E94A12785ED8093BC00D3
:1035E00080913A0290913B02A0913C02B0913D0241
:1035F0000796A11DB11D23E0B695A79597958795D0
:103600002A95D1F72091BC0024FD03C010928302BB
:10361000089540913A0250913B0260913C027091B2
:103620003D02452B462B472B69F30097A105B105B9
:1036300041F02AE22A95F1F700C00197A109B109EA
:10364000E1CF809139020C9440104F925F926F92BB
:103650007F928F929F92AF92BF92CF92DF92EF9222
:10366000FF920F931F93CF93DF938091CE02882315
:1036700009F4F4C08091E9019091EA01892B09F0E5
:1036800073C0A3EDB1E00AE011E0C0E0D1E0CE01EB
:10369000980141E06D917D91F901E080F180F701A1
:1036A000EE0FFF1FE45BFE4F0190F081E02D6E17DF
:1036B0007F0711F0FC014083275F3F4F0196F1E047
:1036C000AF3DBF0739F78091EB019091EC01892B59
:1036D00089F40E94DC15EDEEF1E08991882329F050
:1036E00011821082DE0111971C92329651E0C63091
:1036F000D50799F7CDEED1E092ECC92E92E0D92E04
:10370000F12CE12C2AE0822E912CA12CB12C2881C5
:103710003981F801878190852817390771F48281F2
:103720009381892B09F06CC0F701EE0FFF1FE2595E
:10373000FE4F61E080810E94730688819981F601C5
:10374000219131916F01821793070CF06BC00196A4
:1037500099838883FFEFEF1AFF0A2296075F1F4FB6
:1037600056E0E516F10499F68091E9019091EA019D
:1037700001969093EA018093E9012091DC022111E6
:103780001FC02091DF013091E0018217930708F4F8
:1037900053C01092EA011092E9018091EB019091DF
:1037A000EC018731910508F040C001969093EC013F
:1037B0008093EB018091D0028823F1F10E94631580
:1037C0002091DC028091E9019091EA01223091F58B
:1037D0002091DF013091E0018217930768F1809119
:1037E000EB019091EC018731910530F51092EA01DF
:1037F0001092E90101969093EC018093EB011CC0BB
:103800000E946E25F80142805380712C612CA50125
:1038100094010E94DC2546165706680679060CF4CA
:1038200083CF8BCF1982188295CF1092EC01109222
:10383000EB01C0CF233061F28091E9019091EA0160
:103840000C9760F0CEE6D1E00AE711E0888122967D
:1038500060E00E9473060C171D07C1F7DF91CF913E
:103860001F910F91FF90EF90DF90CF90BF90AF909E
:103870009F908F907F906F905F904F9008951F92D0
:103880000F920FB60F9211242F933F938F939F9314
:10389000AF93BF938091E2029091E302A091E40282
:1038A000B091E5023091E10223E0230F2D3758F566
:1038B0000196A11DB11D2093E1028093E202909335
:1038C000E302A093E402B093E5028091E6029091B6
:1038D000E702A091E802B091E9020196A11DB11D95
:1038E0008093E6029093E702A093E802B093E90286
:1038F000BF91AF919F918F913F912F910F900FBEEC
:103900000F901F90189526E8230F0296A11DB11D58
:10391000D2CF1F920F920FB60F9211242F933F9385
:103920004F935F936F937F938F939F93AF93BF93C7
:10393000EF93FF93E0910801F09109010995FF9140
:10394000EF91BF91AF919F918F917F916F915F9117
:103950004F913F912F910F900FBE0F901F90189590
:103960001F920F920FB60F9211242F933F934F93F4
:103970005F936F937F938F939F93AF93BF93EF93D7
:10398000FF93E0910601F09107010995FF91EF91F6
:10399000BF91AF919F918F917F916F915F914F9167
:1039A0003F912F910F900FBE0F901F9018951F926F
:1039B0000F920FB60F9211242F933F934F935F9363
:1039C0006F937F938F939F93AF93BF93EF93FF93E7
:1039D0008091B6029091B7028093B2008091B902B3
:1039E0009091BA02A091BB02B091BC020196A11DB8
:1039F000B11D8093B9029093BA02A093BB02B09319
:103A0000BC028091B9029091BA02A091BB02B09120
:103A1000BC024091B2025091B3026091B402709125
:103A2000B50284179507A607B70710F18091B80271
:103A300081111EC081E08093B8028091B9029091FB
:103A4000BA02A091BB02B091BC02841B950BA60BDD
:103A5000B70B8093B9029093BA02A093BB02B093C4
:103A6000BC02E091B002F091B10209951092B80247
:103A7000FF91EF91BF91AF919F918F917F916F9146
:103A80005F914F913F912F910F900FBE0F901F901C
:103A900018951F920F920FB60F9211242F933F93F8
:103AA0004F935F936F937F938F939F93AF93BF9346
:103AB000EF93FF938091B900887F803609F44AC064
:103AC000F0F5883209F4A7C018F5803109F49BC0DD
:103AD000B8F4882309F4F9C0883009F494C0FF9140
:103AE000EF91BF91AF919F918F917F916F915F9176
:103AF0004F913F912F910F900FBE0F901F901895EF
:103B0000883109F488C0803251F78093820214C052
:103B1000803409F49DC040F48033B9F38833F9F65A
:103B20008093820285ECB0C0803509F485C0883569
:103B300009F496C0883499F60E94ED1AD0CF8839DE
:103B400009F48CC038F5883729F050F4883611F024
:103B5000803729F683E0809383021092810257C058
:103B6000883809F47BC0803919F0803809F0B7CF64
:103B700080918102803208F071C0E091810281E081
:103B80008E0F809381028091BB00F0E0EF59FD4FD2
:103B900080833DC0803B39F0E0F4803A09F479C07D
:103BA000883A09F09CCF84E08093830210926002EF
:103BB00010925F02E091AC02F091AD020995809104
:103BC0005F0281110FC081E080935F0210923F027B
:103BD00009C0803C09F4A6CF883C09F4A3CF883BF8
:103BE00009F07DCFE091600281E08E0F809360024A
:103BF000F0E0E15CFD4F80818093BB00909160021A
:103C000080915F0229C08091A8028093BB0085EC5F
:103C10008093BC0064CF9091A7028091A602981770
:103C200058F5E091A70281E08E0F8093A702F0E0A3
:103C3000EA57FD4F8081E9CFE091A70281E08E0F26
:103C40008093A7028091BB00F0E0EA57FD4F80838C
:103C50009091A7028091A6029817C8F285E8D8CF64
:103C6000E091A70281E08E0F8093A7028091BB00B4
:103C7000F0E0EA57FD4F80838091850281115CCF8F
:103C800081E08093840284EA8093BC0010928302D6
:103C900026CF85EC8093BC00109283028091810234
:103CA000803230F4E0918102F0E0EF59FD4F108254
:103CB0006091810270E0E091AA02F091AB0281E68E
:103CC00092E00995109281020ACF1092820234CFBD
:103CD0001F93CF93DF93A9E0B3E013961C921E923B
:103CE000129748EE53E060E070E014964D935D93B8
:103CF0006D937C9317978EE891E011969C938E9329
:103D0000E5E1F3E01382128220E830E0358324837A
:103D100080E490E09783868331872087938782872A
:103D2000168A158614861786168681E0858B848B05
:103D30002FEF3FEF338B228B318B208B878B108EB5
:103D4000128E118E80EA91E091838083148E138EFF
:103D5000B68FA58F10A2178E8FEF84A385A386A39D
:103D600087A380A780E89AE1A6E0B0E085AB96AB98
:103D7000A7ABB0AF80EA96E8A1E0B0E081AF92AF28
:103D8000A3AFB4AF80E586AF17AECEEED2E081E14F
:103D900090E09983888384E090E09B838A8383E02A
:103DA00090E09D838C8362E081E10E94A10662E045
:103DB00084E00E94A10688810E944A06182F8A8109
:103DC0000E944A06880F991F812B8E831F821886B6
:103DD00019861A861B861C861D861E861F86188AD3
:103DE000198A1A8ADF91CF911F910895789484B52A
:103DF000826084BD84B5816084BD85B5826085BDE7
:103E000085B5816085BD80916E00816080936E0074
:103E10001092810080918100826080938100809166
:103E20008100816080938100809180008160809317
:103E300080008091B10084608093B1008091B000D7
:103E400081608093B00080917A00846080937A00D2
:103E500080917A00826080937A0080917A008160FC
:103E600080937A0080917A00806880937A00109223
:103E7000C1008FEF93E00E94C625833509F082C010
:103E800090E080E00E94C6258093400181E090E0B0
:103E90000E94C6258093410182E090E00E94C625E1
:103EA0008093CF0260ED72E083E090E00E94E11A1F
:103EB0006CED72E084E090E00E94E11A0AE011E00B
:103EC000C5E0D0E0CE010E94C625F80181938F01A4
:103ED0002196CB33D105B1F762E08EE00E94A106B6
:103EE00062E085E00E94A10660E185E00E94A106F3
:103EF00062E082E00E94A10680E994E190930701CC
:103F000080930601809169008C7F826080936900B4
:103F1000E89ACEE6D1E00AE711E08881229661E0D6
:103F20000E94A1060C171D07C1F7809134039091E0
:103F30003503892B79F10E94F31680911B03909130
:103F40001C036091190370911A03813291050CF0E2
:103F50007DC1AC014052510957FF02C04F5F5F4F16
:103F6000559547956357710977FF02C06F5F7F4F83
:103F700075956795F0E2EF2EF12C03E710E028E14C
:103F800036E07CC10E948B1A63E58FEF93E00E94BC
:103F9000CE25A2CF20911B0330911C03C9010796A7
:103FA00097FD079613E0959587951A95E1F720916F
:103FB000190330911A03AC01429FC001439F900D39
:103FC000529F900D11240E947C269093350380937C
:103FD0003403892B09F0AFCF0E94F316F7E2EF2EDE
:103FE000F12C01E210E025EC3AE042E150E060E320
:103FF00070E085E193E00E94DA0E8AE590E090930C
:1040000022038093210381E090E090932403809326
:10401000230321E02093290320932A03909328036C
:1040200080932703909326038093250382EC9AE0E4
:104030000E94E50C88EB9AE00E94E50C0E94E412D5
:1040400060E273E080E090E00E9409070E9413178D
:104050000E94DC150E94631581E090E0A0E0B0E0D2
:104060008093B2029093B302A093B402B093B502CE
:1040700085E29BE19093B1028093B0028091700041
:104080008E7F809370008091B0008C7F8093B00011
:104090008091B100877F8093B1008091B6008F7DC1
:1040A0008093B600809170008D7F80937000809126
:1040B000B10084608093B1008091B1008C7F8093C7
:1040C000B10086E090E09093B7028093B602109220
:1040D000B9021092BA021092BB021092BC02109266
:1040E000B8028091B6029091B7028093B20080919D
:1040F000700081608093700006E010E0A8EC2A2E2A
:10410000312C44244394512CC2E06C2E712CD4E108
:104110008D2E912CD1E0C9E0E0E0AE2EE0E0BE2E85
:104120008EE00E944A06892B09F08BC28091DB0247
:10413000811187C2D093DB020E943B076093D702B4
:104140007093D8028093D9029093DA028091EE02A4
:104150000E944A06F82E8091F0020E944A06880FBB
:10416000991F8F299091F402891709F4D0C22091E8
:10417000F4024091F5025091F6026091F7027091BD
:10418000F802F4E02F0290011124E82F082E000C11
:10419000FF0BE22BF32BE658FE4FC0800C2C000CDB
:1041A000DD08EE08FF084C0D5D1D6E1D7F1D409360
:1041B000F5025093F6026093F7027093F802809331
:1041C000F4022091F2023091F3022230310509F419
:1041D0009BC22330310509F417C32130310509F0A2
:1041E00096C2833009F093C28091F5029091F60255
:1041F000A091F702B091F80262E0B595A795979566
:1042000087956A95D1F78093F9029093FA02A0936B
:10421000FB02B093FC028091010390910203A091F4
:104220000303B09104038093050390930603A093C6
:104230000703B09308030E943B0760930103709348
:104240000203809303039093040361C2AC014054C2
:10425000510957FF02C04F5F5F4F55954795625513
:10426000710977FF02C06F5F7F4F75956795C0E456
:10427000EC2EF12C02E510E028EF37E085E193E029
:104280000E94DA0E82E0809337038091320390918E
:104290003303892B09F4DFC08CE38093360310923B
:1042A000AF021092AE021092EB021092EA020E944C
:1042B000221087E497E09093AD028093AC0288E4EB
:1042C00097E09093AB028093AA0280913D0387FD13
:1042D0001EC061E00E94A10661E080913D030E9442
:1042E000730661E070E080E090E00E94090760E002
:1042F00080913D030E9473066AE070E080E090E0E8
:104300000E94090761E080913D030E94730680913D
:10431000320390913303892B09F45CC120914A0345
:1043200030914B0340914C0350914D0360E074E297
:1043300084EF90E00E940E26205131094109510975
:1043400056954795379527952093B80064E084E10A
:1043500096E00E94CD1160911B03615085E193E0CE
:104360000E94821264E080E196E00E94CD1180916B
:10437000370360E1813009F064E185E193E00E9458
:10438000821264E08CE096E00E94CD118FE8809369
:1043900052038091190390911A038038910509F016
:1043A00032C180911B0390911C038034910509F068
:1043B0003AC180913703813009F023C18FE980939E
:1043C0005203C2E16AED85E193E00E9482126C2FF4
:1043D00085E193E00E94821261E885E193E00E940A
:1043E00082126091520385E193E00E94821269ED8E
:1043F00085E193E00E9482128091370362E281306E
:1044000009F061EF85E193E00E94821266E086E0A8
:1044100096E00E94CD118091320390913303892B55
:1044200009F405C120914E0330914F034091500390
:104430005091510360E074E284EF90E00E940E26F8
:1044400020513109410951095695479537952795CE
:104450002093B800C1CD61E080913B030E94A1068A
:1044600061E080913C030E94A10680913B03082EED
:10447000000C990BFC01EA55F44FE491F0E0EE0FCB
:10448000FF1FEE56F44F2591349130934303209350
:104490004203FC01E654F44FE491E0934803809119
:1044A0003C03082E000C990BFC01EA55F44FE491F3
:1044B000F0E0EE0FFF1FEE56F44FA591B491B093CC
:1044C0004503A0934403FC01E654F44FE491E093C8
:1044D00049038C91E82BEC93809130039091310348
:1044E000892B09F434C0CFB7F8948091A9028111C7
:1044F00027C0E0EBFBE08491E4ECFBE09491E82F33
:10450000F0E0EE0FFF1FE857F44FA591B491EC9146
:10451000E92321F461E08AE00E94730661E08AE009
:104520000E94A1068CB580618CBD8CB580648CBD69
:1045300061E08DE00E94A10661E08BE00E94A1068F
:104540008091A9028F5F8093A902CFBFBECE61E0A8
:10455000809139030E94A10661E080913A030E9494
:10456000A10680913903082E000C990BFC01EA5535
:10457000F44FE491F0E0EE0FFF1FEE56F44F25915B
:10458000349130933F0320933E03FC01E654F44FF3
:10459000E491E093460380913A03082E000C990BB6
:1045A000FC01EA55F44FE491F0E0EE0FFF1FEE56E8
:1045B000F44FA591B491B0934103A0934003FC0143
:1045C000E654F44FE491E09347038C91E095E8239F
:1045D000EC937BCE8091300390913103892B31F0A5
:1045E00080915303909154030E94D509E0914403B4
:1045F000F0914503908180914903809589238083C0
:10460000A5CE8FECDCCE8036910569F480911B033A
:1046100090911C03409739F480913703813029F43D
:1046200080E180935203C2E0CDCE8FEAFACFE091D1
:104630004403F0914503808190914903892B808345
:10464000CBCC8EE00E944A06892B09F47FCD809165
:10465000DB02882309F47ACD1092DB020E943B072B
:10466000C090D702D090D802E090D902F090DA0240
:10467000DC01CB018C199D09AE09BF09843F51E0D3
:104680009507A105B10578F58091D5029091D602E4
:104690000097A1F48091D3029091D40201968730C3
:1046A000910538F49093D4028093D3020E9413179B
:1046B0004DCD1092D4021092D302F8CF83309105E1
:1046C00068F42091D3023091D402232B09F4A3C1C2
:1046D00001969093D6028093D502E8CF5092D602ED
:1046E0004092D502E3CF803D9740A105B10508F087
:1046F0002DCD8091D5029091D602892B79F310921D
:10470000D6021092D502D2CF882309F46DCDC09085
:10471000F902D090FA02E090FB02F090FC022091A6
:10472000D1023091D2022C153D0559F12C193D09C9
:104730008091D3029091D4024091D5025091D6023B
:10474000009709F0BCC04115510509F07CC080916B
:10475000DC02811110C08091400190914101280F2D
:10476000391F293C310508F461C030924101209283
:1047700040010E9463150E941317D092D202C0928A
:10478000D10285E00E944A06892B29F48091C1025A
:10479000882309F424C185E00E944A06892B09F088
:1047A00032C180E10E94D2069093C0028093BF0282
:1047B0008FE00E94D2069093BE028093BD020E94B9
:1047C0003B07C090DD02D090DE02E090DF02F09067
:1047D000E0026C197D098E099F09613E734984408E
:1047E000910520F00E94F3160E94E4128091DC02F1
:1047F0008250823010F40E946315A114B10409F4B0
:104800008FCC0E94000086CC882319F0833009F0F9
:104810007ECF8091F5029091F602A091F702B091BF
:10482000F802B595A79597958795EDCC243131057C
:1048300028F030934101209340019BCF9092410199
:104840008092400196CF4130510579F48091DC028D
:10485000280F2B3F18F01092DC028DCF243018F473
:104860002093DC0288CF23E0FBCF4230510509F0D2
:1048700082CF8091DC0281117ECF8091D002280FFF
:104880002093D0022F3F61F48091CF02811103C0A9
:104890001092D00270CFC093D0021092CF026BCF93
:1048A0002A3008F468CF8091CF02811105C01092A0
:1048B000D002D093CF025FCFC093D0025CCF41151E
:1048C000510509F50197C89FF001C99FF00D11240A
:1048D000E65FFE4F80819181821B930B8F3F98078B
:1048E00049F4118210828091CE02811144CF0E943E
:1048F000DC1541CF8131910518F491838083F3CF8A
:1049000080E190E0FACF41305105E9F40197C89F6A
:10491000F001C99FF00D1124E65FFE4F8281938163
:10492000280F391F2F3F320719F41382128223CF29
:104930002A30310518F4338322831DCF49E050E03B
:104940005383428318CF4230510519F50197C89F10
:10495000F001C99FF00D1124E65FFE4F858196811D
:10496000280F391F3683258337FF06C084818111C4
:104970000CC016821582FFCE273031050CF4FBCE19
:104980008481811103C0D483F4CF148216830583FC
:10499000F2CE4330510509F0EECE0197C89FF001E9
:1049A000C99FF00D1124E65FFE4F47815085240F0B
:1049B000351F308727832F3F320719F4108617825F
:1049C000DACE880F991FDC01AE53BD4F8D919C91BB
:1049D0002817390708F4CFCE90878783CCCE8091F3
:1049E000DC02811109C00E9463150E946E1480913F
:1049F000CE028D278093CE02D093C1020E948B1AE3
:104A00000E941317CECE8091C102882309F4C9CE2B
:104A10001092C102C6CE019709F060CE7092D60204
:104A20006092D50243CE80EA91E090931603809382
:104A300015038091340390913503009711F00C9485
:104A4000182708958F929F92AF92BF92CF92DF92D4
:104A5000EF92FF92CF93DF93EC01688179818A8195
:104A60009B81611571058105910521F464E279ED61
:104A70008BE597E02DE133EF41E050E00E94DC252B
:104A800049015A019B01AC01A7EAB1E40E94FB2550
:104A90006B017C01ACEEB4EFA50194010E940926E4
:104AA000C60ED71EE81EF91EF7FE06C081E0C81A22
:104AB000D108E10880E8F80AC882D982EA82FB823C
:104AC000C701B6019F77DF91CF91FF90EF90DF9004
:104AD000CF90BF90AF909F908F9008958F929F92AC
:104AE000AF92BF92CF92DF92EF92FF92609142011C
:104AF00070914301809144019091450161157105C8
:104B00008105910521F464E279ED8BE597E02DE1D3
:104B100033EF41E050E00E94DC2549015A019B013E
:104B2000AC01A7EAB1E40E94FB256B017C01ACEE6D
:104B3000B4EFA50194010E940926C60ED71EE81EF7
:104B4000F91EF7FE06C081E0C81AD108E10880E826
:104B5000F80AC0924201D0924301E0924401F092DF
:104B60004501C701B6019F77FF90EF90DF90CF908E
:104B7000BF90AF909F908F90089560934201709383
:104B8000430180934401909345010895F999FECF24
:104B900092BD81BDF89A992780B50895262FF9997D
:104BA000FECF1FBA92BD81BD20BD0FB6F894FA9A10
:104BB000F99A0FBE01960895052E97FB1EF40094F6
:104BC0000E94F32557FD07D00E940E2607FC03D054
:104BD0004EF40C94F32550954095309521953F4F18
:104BE0004F4F5F4F089590958095709561957F4FD9
:104BF0008F4F9F4F08950E943026A59F900DB49F20
:104C0000900DA49F800D911D11240895B7FF0C9461
:104C1000FB250E94FB25821B930B0895A1E21A2E0F
:104C2000AA1BBB1BFD010DC0AA1FBB1FEE1FFF1F50
:104C3000A217B307E407F50720F0A21BB30BE40BA0
:104C4000F50B661F771F881F991F1A9469F76095E7
:104C50007095809590959B01AC01BD01CF010895A1
:104C6000A29FB001B39FC001A39F700D811D1124AD
:104C7000911DB29F700D811D1124911D089597FB08
:104C8000072E16F4009407D077FD09D00E94622603
:104C900007FC05D03EF4909581959F4F089570953F
:104CA00061957F4F08950E943026332312F48A1BAA
:104CB0009B0B0C945D260E943026B7FF0895821B43
:104CC000930B0895AA1BBB1B51E107C0AA1FBB1F72
:104CD000A617B70710F0A61BB70B881F991F5A9588
:104CE000A9F780959095BC01CD010895EE0FFF1FA7
:104CF0000590F491E02D09940F931F93CF93DF93C8
:104D00008230910510F482E090E0E0915703F09139
:104D1000580330E020E0B0E0A0E0309799F421158E
:104D2000310509F44AC0281B390B24303105D8F568
:104D30008A819B816115710589F1FB0193838283CF
:104D4000FE0111C04081518102811381481759072A
:104D5000E0F04817590799F4109761F012960C93F8
:104D6000129713961C933296CF01DF91CF911F912A
:104D70000F9108950093570310935803F4CF211512
:104D8000310551F04217530738F0A901DB019A01B0
:104D9000BD01DF01F801C1CFEF01F9CF90935803B6
:104DA00080935703CDCFFE01E20FF31F81939193C0
:104DB0002250310939832883D7CF20915503309170
:104DC0005603232B41F4209148013091490130933F
:104DD0005603209355032091460130914701211538
:104DE000310541F42DB73EB740914A0150914B0136
:104DF000241B350BE0915503F0915603E217F3079E
:104E0000A0F42E1B3F0B2817390778F0AC014E5F3A
:104E10005F4F2417350748F04E0F5F1F509356031E
:104E200040935503819391939FCFF0E0E0E09CCFB6
:104E3000CF93DF930097E9F0FC013297138212823F
:104E4000A0915703B0915803ED0130E020E0109796
:104E5000A1F420813181820F931F2091550330915D
:104E600056032817390709F061C0F0935603E09301
:104E70005503DF91CF910895EA01CE17DF07E8F5DA
:104E80004A815B819E0141155105B1F7E901FB8320
:104E9000EA8349915991C40FD51FEC17FD0761F4BE
:104EA000808191810296840F951FE90199838883FF
:104EB000828193819B838A83F0E0E0E012968D915A
:104EC0009C9113970097B9F52D913C911197CD01C5
:104ED0000296820F931F2091550330915603281795
:104EE000390739F6309751F510925803109257034D
:104EF000B0935603A0935503BCCFD383C2834081A4
:104F00005181840F951FC817D90761F44E5F5F4F19
:104F100088819981480F591F518340838A819B81E1
:104F2000938382832115310509F0B0CFF0935803A4
:104F3000E09357039ECFFD01DC01C0CF13821282A4
:104F4000D7CF81E090E0F8940C94AD27DC0101C04C
:104F50006D9341505040E0F7089515E0C5EFD5E05E
:104F600004C0FE010E9476262196C63FD107C9F7EC
:104F7000F894FFCF0101010101014907490707002A
:104F8000000000000000000700000000000000001A
:104F90000700000000000000000700000000000003
:104FA00000000700000000000000000700000000F3
:104FB0000000000082000100000000005903800092
:104FC000E8FFF4FFF8FFFAFFFCFFFDFFFEFF010022
:104FD000020003000400050006000700080010009E
:104FE000200006000B0007000A000800090000FF6F
:104FF0000100010000FFFF0000010001FF000000B0
:105000000000B7108A106B14200683107010611016
:1050100000000000130C4A076B14FA0F1E0920064B
:10502000D30EAB0EC70EBB0E4D0F2006D9091514BB
:105030008E08D708F40DD70D5F0D000D0D0A002066
:04504000002B000041
:107800000C94343C0C94513C0C94513C0C94513CE1
:107810000C94513C0C94513C0C94513C0C94513CB4
:107820000C94513C0C94513C0C94513C0C94513CA4
:107830000C94513C0C94513C0C94513C0C94513C94
:107840000C94513C0C94513C0C94513C0C94513C84
:107850000C94513C0C94513C0C94513C0C94513C74
:107860000C94513C0C94513C11241FBECFEFD8E036
:10787000DEBFCDBF11E0A0E0B1E0ECE9FFE702C060
:1078800005900D92A230B107D9F712E0A2E0B1E065
:1078900001C01D92AD30B107E1F70E942D3D0C945F
:1078A000CC3F0C94003C982F959595959595959582
:1078B000905D8F708A307CF0282F295A8091C0000B
:1078C00085FFFCCF9093C6008091C00085FFFCCF60
:1078D0002093C6000895282F205DF0CF982F809127
:1078E000C00085FFFCCF9093C6000895EF92FF92F1
:1078F0000F931F93EE24FF2487018091C00087FD22
:1079000017C00894E11CF11C011D111D81E4E8164B
:1079100082E4F8068FE0080780E0180770F3E09132
:107920000401F091050109958091C00087FFE9CF1E
:107930008091C6001F910F91FF90EF9008950E94D3
:10794000763C982F8091C00085FFFCCF9093C600B5
:1079500091362CF490330CF09053892F089597555D
:10796000892F08951F930E949F3C182F0E949F3CCF
:107970001295107F810F1F9108951F93182F882350
:1079800021F00E94763C1150E1F71F9108951F935A
:10799000182F0E94763C803249F0809103018F5F5E
:1079A000809303018530C1F01F9108958091C0003C
:1079B00085FFFCCF84E18093C6008091C00085FFE5
:1079C000FCCF1093C6008091C00085FFFCCF80E102
:1079D0008093C6001F910895E0910401F091050184
:1079E00009951F9108950E94763C803241F0809164
:1079F00003018F5F80930301853081F008958091AA
:107A0000C00085FFFCCF84E18093C6008091C00058
:107A100085FFFCCF80E18093C6000895E0910401CA
:107A2000F09105010995089540E951E08823A1F0FE
:107A30002D9A28EE33E0FA013197F1F721503040CA
:107A4000D1F72D9828EE33E0FA013197F1F7215064
:107A50003040D1F7815061F708953F924F925F9285
:107A60006F927F928F929F92AF92BF92CF92DF924E
:107A7000EF92FF920F931F93CF93DF93000080E16B
:107A80008093C4001092C50088E18093C10086E015
:107A90008093C2005098589A259A81E00E94143D24
:107AA00024E1F22E9EE1E92E85E9D82E0FE0C02ECA
:107AB00010E1B12EAA24A394B1E49B2EA6E58A2E50
:107AC000F2E57F2EE0E26E2E79E4572E63E5462E36
:107AD00050E5352E0E94763C8033B1F18133B9F107
:107AE000803409F46FC0813409F476C0823409F41B
:107AF00085C0853409F488C0803531F1823521F1A3
:107B0000813511F1853509F485C0863509F48DC0BC
:107B1000843609F496C0843709F403C1853709F423
:107B200072C1863709F466C0809103018F5F80932C
:107B30000301853079F6E0910401F0910501099582
:107B40000E94763C803351F60E94F33CC3CF0E94E2
:107B5000763C803249F78091C00085FFFCCFF092DF
:107B6000C6008091C00085FFFCCF9092C600809136
:107B7000C00085FFFCCF8092C6008091C00085FFC9
:107B8000FCCF7092C6008091C00085FFFCCF609250
:107B9000C6008091C00085FFFCCF5092C600809146
:107BA000C00085FFFCCF4092C6008091C00085FFD9
:107BB000FCCF3092C6008091C00085FFFCCFB09210
:107BC000C60088CF0E94763C863808F4BDCF0E945C
:107BD000763C0E94F33C7ECF0E94763C803809F4CC
:107BE0009CC0813809F40BC1823809F43CC1883942
:107BF00009F48FC080E00E94C73C6CCF84E10E94F2
:107C0000BD3C0E94F33C66CF85E00E94BD3C0E94D3
:107C1000F33C60CF0E94763C809306010E94763C44
:107C2000809307010E94F33C55CF0E94763C80333D
:107C300009F41DC183E00E94BD3C80E00E94C73C66
:107C400049CF0E94763C809309020E94763C809343
:107C5000080280910C028E7F80930C020E94763C79
:107C6000853409F415C18091080290910902892B8D
:107C700089F000E010E00E94763CF801E85FFE4FDA
:107C800080830F5F1F4F80910802909109020817AF
:107C9000190788F30E94763C803209F045CF809125
:107CA0000C0280FF01C16091060170910701660F0F
:107CB000771F7093070160930601A0910802B091AD
:107CC00009021097C9F0E8E0F1E09B01AD014E0F09
:107CD0005F1FF999FECF32BD21BD819180BDFA9A17
:107CE000F99A2F5F3F4FE417F50799F76A0F7B1F4B
:107CF00070930701609306018091C00085FFFCCF5F
:107D0000F092C6008091C00085FFFCCFB092C60003
:107D1000E1CE83E00E94C73CDDCE82E00E94C73CFA
:107D2000D9CE0E94763C809309020E94763C8093D3
:107D300008028091060190910701880F991F909386
:107D40000701809306010E94763C853409F4A6C0A1
:107D500080910C028E7F80930C020E94763C8032D0
:107D600009F0B8CE8091C00085FFFCCFF092C6002C
:107D7000609108027091090261157105B9F140E046
:107D800050E080910C02A82FA170B82FB27011C0E2
:107D9000BB2309F45CC0E0910601F0910701319624
:107DA000F0930701E09306014F5F5F4F46175707B7
:107DB000E8F4AA2369F3F999FECF209106013091E6
:107DC000070132BD21BDF89A90B58091C00085FFB2
:107DD000FCCF9093C6002F5F3F4F30930701209355
:107DE00006014F5F5F4F4617570718F38091C00099
:107DF00085FDE5CE8091C00085FFF8CFE0CE81E023
:107E00000E94C73C67CE0E94763C803209F08CCE3F
:107E10008091C00085FFFCCFF092C6008091C00029
:107E200085FFFCCFE092C6008091C00085FFFCCFAB
:107E3000D092C6008091C00085FFFCCFC092C600E2
:107E40008091C00085FFFCCFB092C60043CEE09188
:107E50000601F091070194918091C00085FFFCCF4D
:107E60009093C6009CCF80E10E94C73C33CE0E9415
:107E7000763C0E94763C182F0E94763C112309F430
:107E800083C0113009F484C08FE00E94C73C22CE29
:107E900080910C02816080930C02E5CE80910C02EF
:107EA000816080930C0259CF809107018823880F4D
:107EB000880B8A2180930B02809106019091070123
:107EC000880F991F90930701809306018091080203
:107ED00080FF09C080910802909109020196909359
:107EE000090280930802F894F999FECF1127E091D6
:107EF0000601F0910701C8E0D1E08091080290915D
:107F00000902103091F40091570001700130D9F34B
:107F100003E000935700E89500915700017001308D
:107F2000D9F301E100935700E89509901990009169
:107F3000570001700130D9F301E000935700E89534
:107F40001395103498F011270091570001700130FB
:107F5000D9F305E000935700E895009157000170B0
:107F60000130D9F301E100935700E895329602976A
:107F700009F0C7CF103011F00296E5CF112480919F
:107F8000C00085FFB9CEBCCE8EE10E94C73CA2CD19
:0E7F900085E90E94C73C9ECDF894FFCF80008B
:00000001FF
